:060000000200E60211A55A
:03000B0002087573
:03001B000200914F
:10003B00C0D0C0E0D228754502754640200A312059
:10004B00091830E908D20AD20878508023D209D295
:10005B00087858C2E8D0E0D0D032A69A08E8B45954
:10006B00087858D20BC208C209C2E8D0E0D0D0320F
:10007B00869A08E8D20EB451067850C208C20AC25A
:10008B00E8D0E0D0D032C0D0C0E0C28E758D4B75B9
:10009B008BFCD28E30B4030200BBE54FB4FF028061
:1000AB000AD54F07754FFFD215D2B3D0E0D0D0325F
:1000BB00D22930080BD54508C208C20AC209C2B3FF
:1000CB00D54613754640D20CD5450B754502E4D287
:1000DB00B3F550120681D0E0D0D032758180C208C2
:1000EB00C20AC209D2B7D2B6D2B5D2B47F787903DD
:1000FB00E4F709DFFB7F1412082EB2B3DFF9C2B3AA
:10010B00754200758D8F758B7FC28ED2A030B40374
:10011B0002079EC2AF75818075400175985A75892B
:10012B001175880175CBFF75CADC75C834C299C2CD
:10013B0098C200C202C201C204C206C2B3C2A2D29A
:10014B009C7541607400120681754200C3D2ABD21C
:10015B008ED2A8D2A9D2B9D2AFC215754FFF30102B
:10016B0005C210121172A298403E300005C2001257
:10017B00022EE580F4F54B300105C2011203CA30A3
:10018B000205C202120549300505C20512042330CF
:10019B000405C2041205F2300605C2061205D8305A
:1001AB001504E412068180B6C29853417FE541B431
:1001BB00600040028003754160E599B4210B7860C3
:1001CB00754160F60541020169B40D08A841F6D2EC
:1001DB0000020169A841F60541020169E4A2B7B327
:1001EB0092E0A2B6B392E1A2B5B392E2F543220834
:1001FB00E6B442097865E6B40D22D20122B4570960
:10020B007865E6B40D16D20222B453107865120647
:10021B00E8F5447867E6B40D03D20522D2062275C1
:10022B004160221201E77860E6B421F3081206E878
:10023B003003ECB543E9C215754FC8D2B308E6B429
:10024B0057028005B451D880A608E6B442030202D7
:10025B00DCB457167867E6B40DC278651206E83041
:10026B0003BAF542120681D20422B4482D7867E610
:10027B00B40DA978651206E83003A120E74D20E6FE
:10028B004A20E54720E44420E341540790038B9335
:10029B004242E542120681D20422B44C2E7867E624
:1002AB00B40D2878651206E830032320E71D20E6FD
:1002BB001A20E51720E41420E311540790038B93C5
:1002CB00F45242E542120681D204220202270202B4
:1002DB002A786DE6B40DF47865E6B43006E542C2D3
:1002EB00E7F542B43106E542D2E7F54208E6B43011
:1002FB0006E542C2E6F542B43106E542D2E6F542E6
:10030B0008E6B43006E542C2E5F542B43106E542F3
:10031B00D2E5F54208E6B43006E542C2E4F542B454
:10032B003106E542D2E4F54208E6B43006E542C2B6
:10033B00E3F542B43106E542D2E3F54208E6B430C8
:10034B0006E542C2E2F542B43106E542D2E2F5429D
:10035B0008E6B43006E542C2E1F542B43106E542A7
:10036B00D2E1F54208E6B43006E542C2E0F542B40C
:10037B003106E542D2E0F542E542120681D2042273
:10038B000102040810204080C37C0833401820145D
:10039B000A7599303099FDC2998021C0E0743012F2
:1003AB000856D0E0801620140A7599313099FDC299
:1003BB00998009C0E07431120856D0E0DCCD2220C0
:1003CB00142A7599243099FDC299E5431205AA7533
:1003DB0099423099FDC299E542120393E54B120302
:1003EB009375990D3099FDC299C2B322D2A2D2B3A3
:1003FB001208427424120856E54312066B7442121B
:10040B000856E542120393E54B120393740D120841
:10041B0056C2A2C214C2B322201417759924309964
:10042B00FDC299E5431205AA7599533099FDC299FE
:10043B008016D2A2D2B31208427424120856E54396
:10044B0012066B7453120856E5445407B40F07E5B4
:10045B0042A2E70204FAB40E07E542A2E60204FA4E
:10046B00B40D07E542A2E50204FAB40C07E542A27B
:10047B00E40204FAB40B07E542A2E30204FAB40A5D
:10048B0007E542A2E20204FAB40907E542A2E1023F
:10049B0004FAB40807E542A2E00204FAB40707E540
:1004AB004BA2E70204FAB40607E54BA2E60204FAF4
:1004BB00B40507E54BA2E50204FAB40407E54BA229
:1004CB00E40204FAB40307E54BA2E30204FAB40214
:1004DB0007E54BA2E20204FAB40107E54BA2E102E5
:1004EB0004FAB40007E54BA2E00204FA0204FA2076
:1004FB00142840137599303099FDC29975990D30B8
:10050B0099FDC299C2B3227599313099FDC2997583
:10051B00990D3099FDC299C2B32240117430120863
:10052B0056740D120856C2A2C214C2B322743112F1
:10053B000856740D120856C2A2C214C2B32220145C
:10054B002E7599243099FDC299E5431205AA759928
:10055B00573099FDC299E542F812075AE54BF87AE4
:10056B000012075A75990D3099FDC299C2B322D268
:10057B00A2D2B31208427424120856E54312066B3A
:10058B007457120856E542F812075AE54BF87A00F1
:10059B0012075A740D120856C214C2A2C2B322F922
:1005AB00C4540F9005C893F5993099FDC299E9543D
:1005BB000F9005C893F5993099FDC29922303132CD
:1005CB003334353637383941424344454620144A93
:1005DB007599243099FDC299E5431205AA75994E78
:1005EB003099FDC29980102014487599243099FDDB
:1005FB00C299E5431205AA7599413099FDC29975C7
:10060B0099433099FDC29975994B3099FDC29975F3
:10061B00990D3099FDC299C2B322D2A2D2B312085E
:10062B00427424120856E54312066B744E12085698
:10063B008011D2A2D2B31208427424120856E54399
:10064B0012066B74411208567443120856744B12FF
:10065B000856740D120856C2B3C2A2C214C2B322FA
:10066B00F9C4540F9005C893120856E9540F90051E
:10067B00C8931208562230A003D2B3E4D2A4C2A767
:10068B00C2A6C2A5A2E092A1C2A4D2A4D2A7A2E103
:10069B0092A1C2A4D2A4C2A7D2A6A2E292A1C2A442
:1006AB00D2A4D2A7D2A6A2E392A1C2A4D2A4C2A7DB
:1006BB00C2A6D2A5A2E492A1C2A4D2A4D2A7A2E5BB
:1006CB0092A1C2A4D2A4C2A7D2A6A2E692A1C2A40E
:1006DB00D2A4D2A7A2E792A1C2A4D2A422E6120668
:1006EB00F5C4FB08E61206F54B22D203B4300374B3
:1006FB000022B43103740122B43203740222B433E6
:10070B0003740322B43403740422B4350374052236
:10071B00B43603740622B43703740722B438037457
:10072B000822B43903740922B44103740A22B44277
:10073B0003740B22B44303740C22B44403740D22D0
:10074B00B44503740E22B44603740F22C2032290E5
:10075B00006412076F90000A12076F9000011207D6
:10076B006F601E227EFF0ECAB58300CA4012C89569
:10077B0082C8CA9583CA50EEC82582C8CA3583CAB7
:10078B004E74302E201408F5993099FDC29922121F
:10079B00085622D2B375818075985A758911758860
:1007AB000075CBFF75CADC75C834758C8F758A7F65
:1007BB0075468075450812081575E800758DFC7532
:1007CB008B66C20D75A901D2ABD28EE41206817570
:1007DB005000755800C20C754C02D2AF300B05128D
:1007EB00080FC20BE580F4F550300C02C20C302818
:1007FB0011D2B330290CC229D54C07754C02C22833
:10080B00C2B380D8E55812068122C0E0E4A2B7B388
:10081B0092E0A2B6B392E1A2B5B392E22430F59B7B
:10082B00D0E022C0E0C0F075F02874E5D5E0FDD52E
:10083B00F0F8D0F0D0E022C0E0C0F075F00A74E51B
:10084B00D5E0FDD5F0F8D0F0D0E0222012FDC0E0CD
:10085B00D20FD211F530753300758CFF758AB0D27B
:10086B008C200FFDD0E0220210A4C28C758CFF757A
:10087B008AACD28CC0D0C0E0C083C0822012E820EA
:10088B001100E5339010002373D082D083D0E0D0D9
:02089B00D03259
:10100000011A0122012E013A01460152015E016AD4
:1010100001760182018A01920192C2A37533010215
:101020000894E530A2E092A3753302020894E530FB
:10103000A2E192A3753303020894E530A2E292A3E1
:10104000753304020894E530A2E392A375330502D8
:101050000894E530A2E492A3753306020894E530C3
:10106000A2E592A3753307020894E530A2E692A3A5
:10107000753308020894E530A2E792A3753309029C
:101080000894D2A375330A020894D2A375330B02D5
:101090000894753300C20FC211C28CD082D083D0A5
:1010A000E0D0D032E5329010AB237301CF01DC01E8
:1010B000EA01F82106211421222130213E214C2170
:1010C000672167216721672167216721672167758C
:1010D0003201A2B25003021167020894753202A2D3
:1010E000B2E53192E0F531020894753203A2B2E51F
:1010F0003192E1F531020894753204A2B2E53192E1
:10110000E2F531020894753205A2B2E53192E3F5B9
:1011100031020894753206A2B2E53192E4F531024B
:101120000894753207A2B2E53192E5F531020894D0
:10113000753208A2B2E53192E6F5310208947532B3
:1011400009A2B2E53192E7F53102089475320AC27C
:101150008CA2B25007D210853135D214C2B3C28CE2
:10116000C212D2A8020894C2B3C28CC212D2A80280
:10117000089453417FE541B460004002800375410B
:1011800060E535B421097860754160F6054122B407
:101190000D09A841F6D20075416022B40A0122A8C7
:1011A00041F6054122758CFF758ADED28C753100BF
:0B11B000C2A8C213D212753200323206
:00000001FF
